:10106B00EA6000D20000010001400160018001A094
:10107B0001C001E002000300039603B603D603F49C
:10108B000400050005180530054805600578059036
:10109B0005A805C0060006140628063C066E068C3D
:1010AB0000FF013F015F017F019F01BF01DF01FFD6
:1010BB0002FF039503B503D503F303FF04FF0517E5
:1010CB00052F0547055F0577058F05A705BF05FFAD
:1010DB0006130627063B066F068B06FFDAD8D7D515
:1010EB00D4D2D0CFCDCBC9C7C6C4C2C0BEBCBAB890
:1010FB00B5B3B1AFADABA8A6A4A2A09D9B99969496
:10110B0092908D8B89878482807E7C7977757371C1
:10111B006F6D6B69676563615F5D5B5957565452C1
:10112B00504F4D4B4A4847454442413F3E3C3B3A6A
:10113B0039373635343231302F2E2D2C2B2A2928A6
:10114B00272625252423222121201F1E1E1D1C1C82
:10115B001B1A1A1919EEECEBEAE9E8E7E5E4E3E10F
:10116B00E0DEDDDBD9D8D6D4D2D0CECCCAC8C6C34C
:10117B00C1BFBCBAB7B5B2B0ADABA8A5A3A09D9B80
:10118B00989592908D8A8785827F7D7A7775726F1D
:10119B006D6A686563615E5C5A575553514F4D4B91
:1011AB004947454342403E3C3B3938363533323173
:1011BB002F2E2D2B2A292827262524232221201FB9
:1011CB001E1D1D1C1B1A1A191818171616150000B0
:1011DB001D0101010500020A0A5A0B000F0D00FA4E
:1011EB000E00020F0132100096110064120132132F
:1011FB0014FA14010215000217010A18010A190A40
:10120B00281A010A1B010A1C0A2823011E240A643E
:10121B002C50782D003C2E05462F001E30006432DA
:10122B005078330000343CFA3501643601643701E1
:10123B0050380A643B00013C00643E003C411450B2
:10124B0042005A430AC8440A3245007847012348F2
:10125B000202500808510A9652143253000B540ADA
:10126B00965601015705465C14325F006464021107
:06127B00650002FAFAFA18
:10004900750B00750A00AE0AAF0BAC08AD09EDC31C
:100059009FEC9E401674FF12137375CF01780B74D1
:100069000126F6500418E436F650DB2290002BE006
:10007900B4AA0D900748E0B43C06E52A4529700367
:1000890002017B900029E4F0A3F075F809AE29AFCD
:100099002A74078E048F05FF1213AFED4C70067496
:1000A9003A900748F07E017F08E56F141213A1907A
:1000B9000027EEF0A3EFF0900029E0FEA3E0FF7423
:1000C9000CD39F74019E5003020176A2F9B3500329
:1000D900020173EF4E700375A382900029E0FEA31D
:1000E900E0FF74016F4E700375A300900029E0FED4
:1000F900A3E0FF74026F4E700BE52A75F002A4FDB0
:10010900ACF08DA3900029E0FEA3E0FF74036F4ECD
:10011900700375A300900029E0FEA3E0FF7403BEFD
:1001290000039F5017900027E0FCA3E0FDED2FFF8F
:10013900EC3EFE9000441213BBE0F5A3900029E0C9
:10014900FEA3E0FFEFB40B09EEB40105741412131A
:1001590073900029E0FEA3E0FFEFB40B07EEB401B2
:100169000375F80D90002912001E0200C090002BA3
:10017900E4F022752C00752B0075F8097E017F08C3
:10018900AC29AD2A1DBDFF011C12002E900021EEE5
:10019900F0A3EFF0AE2BAF2C7411D39F74019E50D6
:1001A9000302027CA2F9B35003020279E52C452B24
:1001B900700375A3D2AE2BAF2C74016F4E7003750B
:1001C900A300AE2BAF2C74026F4E700BE52A75F0AD
:1001D90002A4FDACF08DA3AE2BAF2C74036F4E704F
:1001E9000375A300AE2BAF2C74046F4E700375A377
:1001F90000AE2BAF2C74056F4E700375A300AE2BA8
:10020900AF2C74066F4E700375A300AE2BAF2C7420
:10021900076F4E700375A300AE2BAF2C74086F4E99
:10022900700375A300AE2BAF2C7408BE00039F505A
:100239001A900021E0FCA3E0FDED2FFFEC3EFE90BB
:10024900003F1213BBE5A3F075A300AE2BAF2CEF53
:10025900B41009EEB401057414121373AE2BAF2C4C
:10026900EFB41007EEB4010375F80D782B1213E201
:1002790002019D22C204C205C206C20722752C00D2
:10028900752B0075F809AE2BAF2C7417BE0004D37B
:100299009F500302035CA2F9B35003020359E52CF2
:1002A900452B700375A3D2AE2BAF2C74016F4E7022
:1002B9000375A300AE2BAF2C74026F4E700BE52AA9
:1002C90075F002A4FDACF08DA3AE2BAF2C74036FB7
:1002D9004E700375A300AE2BAF2C74046F4E7003E0
:1002E90075A300AE2BAF2C74056F4E700375A30078
:1002F900AE2BAF2C74066F4E700375A300AE2BAFF7
:100309002C74076F4E700375A300AE2BAF2C7408C5
:100319006F4E700375A300AE2BAF2C7408BE00039B
:100329009F500C90012E1213BBE5A3F075A300AEEC
:100339002BAF2C74166F4E70057414121373AE2BF9
:10034900AF2C74166F4E700375F80D782B1213E2EB
:1003590002028F22C2CF056D22900047E493640602
:10036900600280FE75840175A70075FF8075EF0630
:1003790090002BE4F075C91075A70F75A1C775A773
:100389000075D90075CE0C75A70F75F1FE75F2FFD2
:1003990075F30775F47875A4DA75A5FF75A6077561
:1003A900AE0075AFFF75D48175D5FF75D6FF75D7CA
:1003B900FF75A70075A20175A14775F80975D800E1
:1003C90075D90475DA0975DB0975E60875BC017517
:1003D900BE0475BD6C75BE0775BDA075BE0875BD3B
:1003E9000175BC0075BB1875BC2075BA0875E88025
:1003F90075D11375A70F75E10575E20075C74075CD
:10040900B500C293C294C291C292C287C290E5B5A7
:1004190054EFF5B5E5B554DFF5B5C296C295C2A05E
:10042900C297C2A2C2A1E5B5547FF5B5E5B554BFDF
:10043900F5B5E5B554FBF5B5759700759780740A60
:100449001213737597C0E5975420700280F8758F61
:100459000275A700D2AF75980075A90C75A70F751D
:10046900AB4375ADFB75AC1E75A700758922758EFA
:1004790004758C00758A00C2A9D28CD2ADC2CFD2C4
:10048900CA75D944753E00753D00753A0075390045
:10049900754D00754E00C2997509C875080012009E
:1004A9004975B5F0756E01E56ED39407501A856EDE
:1004B9002A75290012017C75096475080012004922
:1004C900786E740126F650DF752A647529001202C8
:1004D90086752AC8752900900137E0900008F090C8
:1004E9000138E0900009F0900139E090000AF075B8
:1004F9002A66752900120286752AC8752900740AA8
:10050900900060F0740A900063F0740A900099F00A
:100519007404900000F07400900001F0900137E03D
:10052900900002F07403900003F07404900004F04A
:100539007400900005F07400900006F074019000BA
:1005490007F0900138E090000BF0740090000CF077
:10055900740090000DF0740190000EF0740090008A
:100569000FF074FF900010F07400900055F09000A7
:100579007CE0C3943C5006743C90007CF090009958
:10058900E0C3940A5006740A900099F090009BE029
:10059900C3940A5006740A90009BF012027D7559A3
:1005A9000075271975286490001174FFF0A374DC95
:1005B900F0753E00753D00756B00753800753700A4
:1005C900C208757000756100C20D75721E743A908B
:1005D9000748F074FD900749F0C21975740090003E
:1005E90039E4F0754600754500900036E4F0A3F053
:1005F900900054E075F032A4FFAEF08E418F429026
:10060900001BE4F0A3F074FA90002FF0C21CC22181
:10061900A2B6B39200A2B3B39201A2B5B39202A259
:10062900B4B39203755146755200753000752F00A9
:10063900C21B755B00756900755E00755D007562AA
:1006490032756332756400743C90002DF0743C90EF
:10065900002EF075660075670075680090001FE44C
:10066900F0A3F0756A00756501900073E09000349D
:10067900F8E4F0E8A3F0D2B2D2A4D2B0D2B1D2A3B6
:10068900D2A7D2A6D2A5D2B790004AE0D394FE4011
:100699000674FE90004AF090004BE0D394FE4006A9
:1006A90074FE90004BF090004CE0D394FE40067429
:1006B9000A90004CF0900072E0D394FE400674FE5C
:1006C900900072F0900073E0D394FE400674FE909F
:1006D9000073F074FF900088F090008EE0D394FED0
:1006E900400674FE90008EF074FF900091F0900027
:1006F90093E0D3940140067400900093F090009425
:10070900E0D394FE400674FE900094F074FF9000CC
:1007190096F09000A6E0D39464400674649000A615
:10072900F074FF9000A9F09000AAE0D394FE40066F
:1007390074FE9000AAF074FF9000ABF07400900072
:10074900B0F074009000B1F0744D90011FF0746521
:10075900900120F07472900121F07463900122F0ED
:100769007475900123F07472900124F074799001EA
:1007790025F07432900126F07420900127F074540A
:10078900900128F07465900129F0747390012AF0A2
:10079900747490012BF0742090012CF07420900156
:1007A9002DF07400900134F07400900135F074005C
:1007B900900136F0D29CD2EC75CF01A298B35003C8
:1007C9000209DDC298E54E6003020868754E00E52E
:1007D90099B4FF03754D01E599B4FE03754D02E522
:1007E90099B4FD03754D03E599B4FC03754D04E512
:1007F90099B4FA03754D05E599B4FB03754E01E506
:1008090099D394E54007E599C394F0400280168591
:100819009977754E027E017F00E577C394E612133E
:10082900A18E3B8F3C753E00753D00E599D394C779
:100839004007E599C394E64002801F859977754E74
:100849000374E5C39577F53C753B00AE3BAF3C902F
:10085900106F121362783D1213D0D2990209DDE5A7
:100869004EB401028003020945AE3DAF3E900048F7
:100879001213BBE599F0783D1213E2AE3DAF3EEF9E
:10088900B40106EEB407028003020945900748E067
:10089900B43C02800302093FC29C12027D900038D9
:1008A9007401F0743C900748F0900038E01475F03A
:1008B90007A4FFAEF08F6E756F01E56FD3940750F3
:1008C90023E56F256EF52A75290074AA90002BF08F
:1008D900120075750964750800120049786F740172
:1008E90026F650D67599FB7402900038F0743C9046
:1008F9000748F0900038E01475F007A4FFAEF08FB8
:100909006E756F01E56FD394075023E56F256EF57A
:100919002A75290074AA90002BF0120075750964D4
:10092900750800120049786F740126F650D6752AA9
:10093900C8752900D29C754E00754D00E54EB4026C
:100949004CE53E453D700685993A753900AE3DAF97
:100959003E74016F4E701BAC39AD3AAA3BAB3CED0E
:100969002BFBEC3AFA8A068B079000481213BBE579
:1009790099F0783D1213E2AE3DAF3E74026F4E70AE
:100989000C12027D857799754E00754D00E54EB4C0
:100999000342AE3DAF3E9000481213BBE599F07893
:1009A9003D1213E2AE3DAF3EAC3BAD3C8F028E0330
:1009B9008C068D079010AB121362E493F9740193BE
:1009C900FEEAD39EEB99400C12027D857799754E0C
:1009D90000754D00E54D6006A299B3B34003020BC3
:1009E9003EC299E54DB4011FAE3DAF3E90000012E5
:1009F90013BBE0F599783D1213E2AE3DAF3E741199
:100A09006F4E7003754D00E54DB40203856599E598
:100A19004DB4031DAE3DAF3E9000481213BBE0F547
:100A290099EFB40107EEB40703754D00783D121331
:100A3900E2E54DB404028003020B1DE53E453D701D
:100A490003853099AE3DAF3E74016F4E7003855BEF
:100A590099AE3DAF3E74026F4E7003855E99AE3D0F
:100A6900AF3E74036F4E7003856299AE3DAF3E741D
:100A7900046F4E7003856499AE3DAF3E74056F4EA9
:100A89007003856699AE3DAF3E74066F4E7003855F
:100A99006799AE3DAF3E74076F4E7003856899AE96
:100AA9003DAF3E74086F4E7006900020E0F599AE98
:100AB9003DAF3E74096F4E700690002FE0F599AE78
:100AC9003DAF3E74096F4E700590002FE4F0AE3DC6
:100AD900AF3E740A6F4E7003856999AE3DAF3E749F
:100AE9000B6F4E7003856399AE3DAF3E740C6F4E2C
:100AF9007003856A99AE3DAF3E740D6F4E700375F4
:100B090099FC783D1213E2AE3DAF3E740E6F4E7004
:100B190003754D00E54DB4051CAE3DAF3E9011D9AE
:100B29001213BBE493F59974A76F4E7003754D00CA
:100B3900783D1213E2E54EB401030207C1C2CA7E31
:100B4900107F00E56D1213A1E5CD75F010A4FDAC81
:100B5900F0EF2DFDEE3CFCE5CC75F01084FF7E0036
:100B6900ED2FFFEC3EFE8E278F28D2CAA2B3400696
:100B7900E5B554DFF5B5A2B3B34006E5B54420F5B4
:100B8900B5A2B54006E5B5547FF5B5A2B5B34006A3
:100B9900E5B54480F5B5A2B44006E5B554BFF5B551
:100BA900A2B4B34006E5B54440F5B5A2B63000019C
:100BB900B35003020C6CA2B6300001B35003020C0F
:100BC9006CA2B6300401B35003020C59E5B554FBCD
:100BD900F5B5E55A7060E5284527601AAE27AF28B4
:100BE900740112139390106BE493FC740193FD123A
:100BF90012818E2F8F30AE2FAF307428BE00039F25
:100C09005010E5612FFF50010E74011213938E2FBE
:100C19008F30853061900099E0A82FB8000DD395E9
:100C2900304008E53090002CF08009900099E014DC
:100C390090002CF08002155AC2CA75CD0075CC00FF
:100C4900756D00752801752700D2CAA204B39200F8
:100C5900A204B330B601B3400AE5B54404F5B5A220
:100C690004920090001112001E900011E0FEA3E012
:100C7900FFEFB47006EEB417028003020E3B90003A
:100C890011E4F0A3F00552E552B40A30E5B554FE7B
:100C9900F5B5C2A2C2A0C296E5B554F7F5B5C2939F
:100CA900C291C287E5B554EFF5B5E5B554FDF5B583
:100CB900C2A1C297C295C294C292C290E552B4141D
:100CC90030E5B54401F5B5D2A2D2A0D296E5B54436
:100CD90008F5B5D293D291D287E5B54410F5B5E5BB
:100CE900B54402F5B5C2A1C297C295C294C292C2D7
:100CF90090E552B41E30E5B554FEF5B5C2A2C2A0C6
:100D0900C296E5B554F7F5B5C293C291C287E5B568
:100D190054EFF5B5E5B554FDF5B5D2A1D297D29505
:100D2900D294D292D290E552B42830E5B554FEF56A
:100D3900B5C2A2C2A0C296E5B554F7F5B5C293C231
:100D490091C287E5B554EFF5B5E5B554FDF5B5C2E2
:100D5900A1C297C295C294C292C290E552B43230F0
:100D6900E5B54401F5B5C2A2C2A0C296E5B554F7EE
:100D7900F5B5C293C291D287E5B554EFF5B5E5B59E
:100D890054FDF5B5C2A1C297C295C294C292D29040
:100D9900E552B43C30E5B554FEF5B5D2A2C2A0C2C5
:100DA90096E5B554F7F5B5C293D291C287E5B55426
:100DB900EFF5B5E5B554FDF5B5D2A1C297C295C217
:100DC90094D292C290E552B44630E5B554FEF5B5D9
:100DD900C2A2D2A0C296E5B554F7F5B5D293C29195
:100DE900C287E5B554EFF5B5E5B554FDF5B5C2A132
:100DF900D297C295D294C292C290E552B45033E5CB
:100E0900B554FEF5B5C2A2C2A0D296E5B54408F51F
:100E1900B5C293C291C287E5B554EFF5B5E5B554AE
:100E2900FDF5B5C2A1C297D295C294C292C290757E
:100E39005200E56BB40A03756B00E56BC3940A4075
:100E490003021036A2EDB35003021036C2EDE56B72
:100E5900701E7E017F00E5BE1213A1E5BD2FFF5074
:100E6900010E8E318F3274041213938F5B75BB1888
:100E7900E56BB401207E017F00E5BE1213A1E5BD3B
:100E89002FFF50010E8E318F3274041213938E5D31
:100E99008F5E75BB19E56BB402237E017F00E5BE49
:100EA9001213A1E5BD2FFF50010E8E318F32742927
:100EB9008E048F05FF1213838D6275BB13E56BB426
:100EC900031E7E017F00E5BE1213A1E5BD2FFF5071
:100ED900010E8E318F3274041213938F6375BB1711
:100EE900E56BB404667E017F00E5BE1213A1E5BD82
:100EF9002FFF50010E74041213938E318F3290001C
:100F09002DE0601290002DE0149010E793A831B8FD
:100F1900000695324002800690002DE014F0900002
:100F29002DE0C39477501390002DE0049010E793BF
:100F3900A831B80005D395325002800690002DE003
:100F490004F090002DE0F56475BB16E56BB40566F9
:100F59007E017F00E5BE1213A1E5BD2FFF50010EF2
:100F690074041213938E318F3290002EE060129028
:100F7900002EE01490116093A831B8000695324014
:100F890002800690002EE014F090002EE0C39477C2
:100F9900501390002EE00490116093A831B8000519
:100FA900D395325002800690002EE004F090002E76
:100FB900E0F56675BB1FE56BB406287E017F00E589
:100FC900BE1213A1E5BD2FFF50010E8E318F327471
:100FD900091213A174E68E048F05FF1213838D681D
:100FE90075BB15E56BB4071E7E017F00E5BE1213C4
:100FF900A1E5BD2FFF50010E8E318F3274041213FB
:10100900938F6775BB14E56BB4081E7E017F00E5FD
:10101900BE1213A1E5BD2FFF50010E8E318F327420
:10102900041213938F6975BB1A056BD2ECAE27AF07
:1010390028EFD394DCEE94FF4025755146755A028A
:10104900753000752F0075610090001FE4F0A3F062
:1010590075280075270075CD0075CC00756D0002E7
:0210690007C1BD
:10136200EF2F500205832582F582E5833E2EF58319
:011372002258
:0913D000E493F608740193F6227F
:0813E2000806B60002180622FD
:0D001E00A3E004F070061213C6E004F02207
:0E139300048007C3CE13CECF13CFD5E0F622D1
:10128100BC000FBE0008ED8FF084FFADF022E4FE3C
:10129100FF22BE000DEF60FE54F0606F20E70302F5
:1012A1001337EAC0E0EBC0E078017A0075F001EE97
:1012B10020E710EF25E0FFEE33FE0AC5F023C5F06D
:1012C10030E7F0EA5407F9096A7A007B0060010807
:1012D100C3EC9E40167004ED9F4010ED9FFDEC9E07
:1012E100FCE5F0CA4ACA03F5F08005E5F003F5F024
:1012F100C3EE13FEEF13FFD9D77908CACBCAD8D0F2
:10130100EAFEEBFFD0E0FBD0E0FA22EC8FF084FCA8
:10131100ED54F045F0C48FF084FEEDC454F045F077
:10132100C48FF084FDEEC4FE54F02DFFEE540F3C4B
:10133100FEADF07C0022790078008FF0EC7E082071
:10134100E70DC3CD33CD33C933C9C833C8DEF0840B
:1013510049F9E5F08FF0BE00E6FD7C00E9FFE8FE0B
:011361002269
:0E13A100F88FF0A4FFE5F0CE88F0A42EFE2217
:10002E00EF8DF0A4F9A8F0EF8CF0A428F8EE8DF087
:06003E00A428FEE9FF22E8
:10137300600D782B02137D007830D8FED5E0F8227B
:10138300EEC0E07E00121281EFFDEEFCD0E0FE2203
:0C13AF00EEC0E07E00121281D0E0FE22B1
:03002B00020003CD
:030000000213D90F
:0913D90075817D75D000020362EC
:1013BB00E5822FF582E5833EF583220582D58202F5
:0513CB001583158222CC
:10000300C0E0C0F0C083C082C0D075D00012035DD1
:0B001300D0D0D082D083D0F0D0E032FB
:00000001FF
